:100000000C945B000C9481000C9481000C94810092
:100010000C9481000C9481000C9481000C9481005C
:100020000C9481000C9481000C9481000C9481004C
:100030000C9481000C9481000C9481000C9481003C
:100040000C9488010C9481000C946A030C94810038
:100050000C9481000C9481000C9481000C9481001C
:100060000C9481000C9481008701000000070002BD
:10007000010000030406000000000000000001026F
:100080000408102040800102040810200102040826
:100090001020040404040404040402020202020204
:1000A0000303030303030000232629000025282B54
:1000B000000024272A0011241FBECFEFD4E0DEBFAA
:1000C000CDBF11E0A0E0B1E0ECECF9E002C005909A
:1000D0000D92A630B107D9F711E0A6E0B1E001C05A
:1000E0001D92A139B107E1F710E0CAE6D0E004C0E3
:1000F0002297FE010E94E204C836D107C9F70C948A
:10010000B7000C94000061E0809100010E943E0263
:1001100040E855E260E070E088E091E00E94C400B1
:10012000089588E091E00E94CD00909307018093AC
:1001300006012FEF8F3F9207C9F081369105B1F488
:1001400062E071E088E091E00E94D70061E0809178
:1001500000010E94A50268EC70E080E090E00E943F
:10016000C50160E0809100010E94A5020895CFEFD3
:10017000D4E0DEBFCDBF0E94F4010E9483000E9444
:100180009100FDCF08950895CB01BA010E94F002BD
:1001900008950E943103992708950E94420308950B
:1001A0000E9461030895862F0E94A8030895CB0141
:1001B0000E94AF030895862F0E94A80308950F930D
:1001C0001F938C016DE00E94D3006AE0C8010E9479
:1001D000D3001F910F9108950F931F938C010E94DC
:1001E000D300C8010E94DF001F910F9108950F9363
:1001F0001F938C010E94D700C8010E94DF001F914D
:100200000F9108950F931F938C010E94DB00C8018A
:100210000E94DF001F910F910895CB01BA0133278F
:10022000442755270E94BC0308952AE00E940D012F
:1002300008950F931F938C010E941501C8010E941D
:10024000DF001F910F910895AB01662777270E9469
:1002500015010895EF92FF920F931F93CF93DF93B1
:10026000EC017A018B0177FF0BC06DE20E94D30095
:1002700010950095F094E094E11CF11C011D111DF6
:100280002AE0B801A701CE010E940D01DF91CF91B4
:100290001F910F91FF90EF9008950F931F938C0182
:1002A0000E942A01C8010E94DF001F910F9108954A
:1002B0002115310521F4642F0E94D30008952A30BE
:1002C000310519F40E942A0108950E940D01089534
:1002D0000F931F938C010E945801C8010E94DF00F8
:1002E0001F910F910895AB01662757FD6095762FFA
:1002F0000E942A0108950F931F938C010E9473019D
:10030000C8010E94DF001F910F910895089508957C
:100310001F920F920FB60F9211248F939F93AF935A
:10032000BF9380910D0190910E01A0910F01B091AA
:1003300010010196A11DB11D80930D0190930E0136
:10034000A0930F01B0931001BF91AF919F918F9136
:100350000F900FBE0F901F90189560910D01709136
:100360000E0180910F019091100127E0660F771F19
:10037000881F991F2A95D1F72DE730E040E050E023
:100380000E948F04CA01B9010895AF92BF92CF9223
:10039000DF92EF92FF920F931F935B016C010E941B
:1003A000AD017B018C010E94AD016E197F09800BAC
:1003B000910B6A157B058C059D05A8F31F910F9184
:1003C000FF90EF90DF90CF90BF90AF90089501978E
:1003D00051F0880F991F880F991F02972FB7F89433
:1003E0000197F1F72FBF0895789410920D011092A4
:1003F0000E0110920F011092100184B5826084BD2D
:1004000084B5816084BD85B5826085BD85B5816018
:1004100085BDEEE6F0E0808181608083E1E8F0E078
:10042000808182608083808181608083E0E8F0E069
:10043000808181608083E1EBF0E080818460808353
:10044000E0EBF0E0808181608083ECE7F0E0808188
:100450008F778083808180648083EAE7F0E0808109
:1004600084608083808182608083808181608083DA
:100470008081806880831092C1000895282F3327DF
:10048000C90182589F4FFC0194912E563F4FF901AC
:100490008491882381F0E82FFF27E055FF4FE491F6
:1004A000FF27662329F4808190958923808308950E
:1004B0008081892B80830895482F5527CA0186594A
:1004C0009F4FFC012491CA0182589F4FFC019491D7
:1004D0004E565F4FFA0134913323A1F1222331F1BB
:1004E000233021F4809180008F7705C0243031F4CF
:1004F000809180008F7D8093800018C0213019F496
:1005000084B58F7704C0223021F484B58F7D84BDFB
:100510000DC0263021F48091B0008F7705C02730C0
:1005200029F48091B0008F7D8093B000E32FFF27E6
:10053000EA55FF4FE491FF278081892319F081E07C
:1005400090E0089580E090E00895482F5527CA0173
:1005500086599F4FFC012491CA0182589F4FFC018C
:1005600094914E565F4FFA0134913323C1F1222307
:1005700031F1233021F4809180008F7705C0243041
:1005800031F4809180008F7D8093800018C02130ED
:1005900019F484B58F7704C0223021F484B58F7D9F
:1005A00084BD0DC0263021F48091B0008F7705C046
:1005B000273029F48091B0008F7D8093B000E32F25
:1005C000FF27E555FF4FE491FF27662329F480813B
:1005D00090958923808308958081892B8083089555
:1005E000EF92FF920F931F937B018C0122E030E08A
:1005F00040E050E00E94B104205C3D4B404F5F4F13
:10060000CA01B901A80197010E94B10421503040EC
:1006100040405040BB2757FDBA95A52F942F832FFC
:100620002F5F3F4F4F4F5F4F8093C5002150209366
:10063000C400E1ECF0E0808180618083808188608B
:1006400080838081806880831F910F91FF90EF905D
:100650000895982F8091C00085FFFCCF9093C6002D
:10066000089580910B0190910C0120910901309126
:100670000A01821B930B80589F4F60E870E00E9434
:100680007C0408954091090150910A0180910B0169
:1006900090910C018417950719F48FEF9FEF08953F
:1006A000FA01EF5EFE4F2081CA01019660E870E01A
:1006B0000E947C0490930A0180930901822F99275C
:1006C00008958091090190910A0190930C01809303
:1006D0000B0108951F920F920FB60F9211242F93C2
:1006E0003F934F935F936F937F938F939F93AF93BA
:1006F000BF93EF93FF934091C600E0910B01F091FF
:100700000C01CF01019660E870E00E947C049C011E
:100710008091090190910A012817390739F0EF5E9D
:10072000FE4F408330930C0120930B01FF91EF911A
:10073000BF91AF919F918F917F916F915F914F91F9
:100740003F912F910F900FBE0F901F901895089515
:100750000E94290308958AE00E94A8030895CF9378
:10076000DF93EC0103C021960E94A80388818823AF
:10077000D1F7DF91CF9108952F923F924F925F92E0
:100780006F927F928F929F92AF92BF92CF92DF92A1
:10079000EF92FF920F931F93CF93DF93CDB7DEB706
:1007A000A0970FB6F894DEBF0FBECDBF6B017C01E2
:1007B00019012A01611571058105910521F480E374
:1007C0000E94A8034BC06624772443015E0108946D
:1007D000A11CB11C8501060D171DC701B601A201A0
:1007E00091010E948F04F80160830894611C711CC0
:1007F000811C911CC701B601A20191010E948F04C6
:1008000069017A01211531054105510519F7730177
:100810000894E108F108EA0CFB1CAA24BB2465013A
:1008200011C0F70180818A3010F4805D01C0895CBD
:100830000E94A8030894A108B108C108D10808942F
:10084000E108F10888279927DC0186199709A8098A
:10085000B909A816B906CA06DB0619F7A0960FB69D
:10086000F894DEBF0FBECDBFDF91CF911F910F91E6
:10087000FF90EF90DF90CF90BF90AF909F908F90C0
:100880007F906F905F904F903F902F900895EF92E0
:10089000FF920F931F937B018C0197FF0BC08DE29A
:1008A0000E94A80310950095F094E094E11CF11CBF
:1008B000011D111D2AE030E040E050E0C801B70101
:1008C0000E94BC031F910F91FF90EF90089520E1CB
:1008D00030E040E050E00E94BC03089528E030E0A2
:1008E00040E050E00E94BC03089522E030E040E088
:1008F00050E00E94BC03089597FB092E07260AD0FA
:1009000077FD04D049D006D000201AF47095619587
:100910007F4F0895F6F7909581959F4F0895A1E236
:100920001A2EAA1BBB1BFD010DC0AA1FBB1FEE1F69
:10093000FF1FA217B307E407F50720F0A21BB30BB4
:10094000E40BF50B661F771F881F991F1A9469F730
:1009500060957095809590959B01AC01BD01CF018C
:10096000089597FB092E05260ED057FD04D0D7DF3A
:100970000AD0001C38F450954095309521953F4F92
:100980004F4F5F4F0895F6F790958095709561955C
:100990007F4F8F4F9F4F0895AA1BBB1B51E107C08C
:1009A000AA1FBB1FA617B70710F0A61BB70B881FFF
:1009B000991F5A95A9F780959095BC01CD0108958E
:0C09C000EE0FFF1F0590F491E02D09944C
:0609CC000D004142430052
:00000001FF
